:020000040800F2
:1000000000040020E1010008310F0008350F00084E
:10001000890F0008350F00085D0F0008E301000894
:10002000E3010008E3010008E30100086528000877
:10003000E3010008E3010008E3010008E301000810
:10004000E3010008E3010008E3010008E301000800
:10005000E3010008E3010008AD380008D9380008C2
:1000600005390008313900085D390008E30100084E
:10007000E3010008E3010008E3010008E3010008D0
:10008000E3010008E3010008E3010008E3010008C0
:10009000E3010008E3010008E301000889390008D2
:1000A000E3010008E3010008E3010008E3010008A0
:1000B000E3010008E3010008E3010008E301000890
:1000C000E3010008E3010008E3010008E301000880
:1000D000E3010008E3010008E3010008E301000870
:1000E000F1390008E3010008E3010008E30100081A
:1000F000E3010008E3010008E3010008E301000850
:10010000E3010008E3010008BD360008E301000830
:10011000E301000819100008E3010008E3010008EA
:10012000E3010008E3010008E3010008E30100081F
:10013000E3010008E3010008E3010008E30100080F
:10014000E3010008E3010008E3010008512F000863
:10015000E3010008E3010008E3010008E3010008EF
:10016000E3010008E3010008E3010008E3010008DF
:10017000E3010008E3010008E3010008E3010008CF
:10018000E3010008E3010008E3010008E3010008BF
:10019000E3010008E3010008E3010008E3010008AF
:1001A000E3010008E3010008E3010008E30100089F
:1001B000E3010008E3010008E3010008E30100088F
:1001C000E3010008E3010008E3010008E30100087F
:1001D000E3010008E3010008E3010008E30100086F
:1001E00002E000F000F8FEE772B6394880F30888B4
:1001F000384880F3098838484EF60851CEF200019D
:10020000086040F20000CCF200004EF63471CEF2ED
:1002100000010860BFF34F8FBFF36F8F40F2000003
:10022000C0F2F0004EF68851CEF200010860BFF334
:100230004F8FBFF36F8F4FF00000E1EE100A4EF6C4
:100240003C71CEF200010860062080F31488BFF3F1
:100250006F8F02F045FB03F0C7F94FF055301F498F
:100260001B4A91423CBF41F8040BFAE71C49194A6A
:1002700091423CBF41F8040BFAE71A491A4A1B4B5A
:100280009A423EBF51F8040B42F8040BF8E70020F5
:100290001749184A91423CBF41F8040BFAE702F0B3
:1002A00023FB03F0FDF9144C144DAC4203DA54F86F
:1002B000041B8847F9E700F03FF8114C114DAC42A0
:1002C00003DA54F8041B8847F9E702F00BBB00007F
:1002D000000400200024002000000008000000208E
:1002E00000040020983E000800240020282400205C
:1002F00028240020C4340020E0010008E0010008A8
:10030000E0010008E00100082DE9F04F2DED108A12
:10031000C1F80CD0C3689D46BDEC108ABDE8F08FD3
:10032000002383F311882846A047002001F018FF1E
:1003300001F038FE00DFFEE770B5214C6FF00203DC
:1003400023700323002563706FF03F061F23A57001
:10035000E57025716571A571E57125726672A372EC
:10036000E57200F0B3FC20B10F2325726672A37210
:10037000E57202F049FA044602F06EFA0546D8B971
:10038000104B9C421AD001339C4218BF054641F2E3
:10039000883404BF01250024002002F03FFA0DB18B
:1003A00000F05AF800F070FD00F0BEFB204600F0AF
:1003B000B1F800F051F8F9E70024EDE70446EBE767
:1003C00028240020010007B008B500F02BFBA0F1A5
:1003D00020035842584108BD07B5054B02211B8830
:1003E000ADF8043001A800F089FB03B05DF804FB10
:1003F000D83A000810B5202383F311881248C36847
:100400000BB101F033FF0023104A0F484FF47A710B
:1004100001F0F0FE002383F311880D4C236813B123
:100420002368013B2360636813B16368013B636029
:10043000084B1B7833B9636823B9022000F08AFCAB
:100440003223636010BD00BF34240020F503000890
:10045000502500204824002010B5254B254953F88D
:10046000042F013200D110BD8B42F8D1224C234B16
:1004700022689A423AD9224B9B6803F1006303F544
:1004800080439A4232D2002000F068FB1D4B0220CC
:10049000187000F051FC1C4B1A6C00221A64196E83
:1004A0001A66196E596C5A64596E5A665A6E5A69B0
:1004B00042F080025A615A6922F080025A615A69F8
:1004C0001A6942F000521A611A6922F000521A6148
:1004D0001B6972B60D4A0E4B13601B6822682021FF
:1004E00081F311889D4683F30888104710BD00BF33
:1004F000FC3F00081C40000804400008FF3F0008C3
:1005000028240020482400200038024008ED00E0A4
:10051000004000082DE9F04F99B0B34C0190202223
:10052000FF2110A8A66800F051FCB04A1378A3463A
:10053000A3B9AF480121C3601170202383F3118850
:10054000C3680BB101F092FE0023AA4AA8484FF4F9
:100550007A7101F04FFE002383F31188019B13B1E0
:10056000A54B019A1A60A54AA349019F0292002354
:1005700013704B6099461C461D469846012000F0BA
:10058000DBFB002F00F012829B4B1B68002B40F01E
:100590000D8219B0BDE8F08F0220FFF715FF00288B
:1005A00040F0FB81019BB9F1000F08BF1F46944B3F
:1005B0001B88ADF82C3002210BA800F09FFADDE774
:1005C0004FF47A7000F02EFA031E0393EADB022048
:1005D000FFF7FAFE82460028E4D0039B581E042849
:1005E00000F2DD81DFE800F0030E1114170018A8F7
:1005F000052340F8343D042100F080FA54464FF0C2
:10060000000856E004217848F6E704217D48F3E726
:1006100004217D48F0E71C24204600F0A1FA0434B0
:100620000B9004210BA800F069FA2C2CF4D1E5E71B
:10063000002DB7D0002CB5D00220FFF7C5FE05462F
:10064000002800F0AF8101206C4C00F087FA0220F6
:10065000207000F071FB4FF000095FFA89FA5046F4
:1006600000F08CFA074658B1504600F097FA09F1AD
:1006700001090028F1D12C46A9460027634B97E7D2
:1006800001230220237000F04BFB3E46DBF80830CC
:100690009E4206D2304600F063FA0130EBD10436B8
:1006A000F4E7029B00261E70534BA9465E602C4661
:1006B000374600F0DFFB15B1002C18BF0027FFF70D
:1006C0008BFE5BE7002D3FF46DAF002C3FF46AAF6B
:1006D000029B0220187000F02FFB322000F0A2F9DC
:1006E000B0F1000AC0F25E811AF0030540F05A81B1
:1006F000DBF8082006EB0A03934200F25381BAF5B7
:10070000807F00F24F8155450DDA4FF47A7000F08A
:1007100089F90490049B002BC0F244813C4A049B5D
:10072000AB540135EFE7C820FFF74EFE0546002821
:1007300000F038811F2E11D8C6F12004544528BF7F
:10074000544610AB26F0030022463149184400F00D
:1007500013FB2246FF212E4800F038FB4FEAAA0A7D
:100760005FFA8AF22A49304600F038FB0446002836
:1007700000F01A8106EB8A0605469AE70220FFF789
:1007800023FE00283FF40EAF00F02EFA00283FF4BD
:1007900009AF4FF0000A5346DBF8082092451CD2FF
:1007A000BAF11F0F12D8109A01320FD02AF00302AB
:1007B00018A90A4452F8202C0B92184604220BA9BF
:1007C00000F0F6FB0AF1040A0346E5E750460393FE
:1007D00000F0C6F9039B0B90EFE718A8042140F83E
:1007E0004C3D00F08BF964E7282400204C250020C4
:1007F00034240020F5030008502500204824002060
:10080000DA3A00082C24002030240020DC3A0008CA
:100810004C24002018A8002340F8343D642100F047
:1008200039F900287FF4BEAE0220FFF7CDFD002885
:100830003FF4B8AE0B9800F0C3F918AB43F8480D7D
:1008400004211846CDE718A8002340F8343D642160
:1008500000F020F900287FF4A5AE0220FFF7B4FDD8
:1008600000283FF49FAE0B9800F0B8F918AB43F89E
:10087000440DE5E70220FFF7A7FD00283FF492AE04
:1008800000F0C2F918AB43F8400DD9E70220FFF79A
:100890009BFD00283FF486AE0BA9142000F0BAF9A6
:1008A000824618A8042140F83CAD00F027F95146D3
:1008B0000BA896E7322000F0B5F8B0F1000AFFF679
:1008C00071AE1AF0030F7FF46DAEDBF808200AEB6F
:1008D000080393423FF666AE0220FFF775FD00283D
:1008E0003FF460AE2AF0030AC244D0453FF4E1AEC3
:1008F000404600F035F904210A900AA800F0FEF8FD
:1009000008F10408F1E74FF47A70FFF75DFD002865
:100910003FF448AE00F068F900283FF4AFAE109BFA
:1009200001330CD0082210A9002000F057FA00284B
:100930003FF4A4AE2022FF2110A800F047FAFFF7F1
:100940004BFD374801F012FC23E6002D3FF42AAEA0
:10095000002C3FF427AE18A8002340F8343D642152
:1009600000F098F8824600287FF41CAE0220FFF7C2
:100970002BFD00283FF416AE0390FFF72DFD41F24A
:10098000883001F0F3FB0B9800F0B2FA00F072FA35
:10099000039B57461C461D46F0E5054689E64FF089
:1009A0000008FFE52546FDE52C4667E6002000F03F
:1009B00039F80490049B002BFFF6E3AD012000F012
:1009C000AFF9049B213B122B3FF6D8AD01A252F8A0
:1009D00023F000BF99050008C10500083106000892
:1009E0007D0500087D0500087D050008C506000896
:1009F000B50800087D07000815080008470800082A
:100A0000750800087D0500088D0800087D050008B0
:100A100007090008B30600087D0500084B09000817
:100A2000A08601002DE9F34702AE00244FF47A7549
:100A300006F8014D144FDFF85880454397F9003010
:100A40005A1C5FFA84F901D0A34212D158F824004D
:100A500003680122D3F820A031462B46D047012855
:100A600007D10A4B9DF8070083F8009002B0BDE85B
:100A7000F0870134022CE1D14FF4FA7001F076FBDB
:100A80004FF0FF30F2E700BF00240020982500203F
:100A9000303B00082DE9F0474FF47A75144FDFF82A
:100AA000588006464D43002497F900305A1C5FFADF
:100AB00084F901D0A34210D158F82400036804221D
:100AC000D3F820A031462B46D047042805D1094B46
:100AD00083F800900020BDE8F0870134022CE3D1B8
:100AE0004FF4FA7001F042FB4FF0FF30BDE8F087A1
:100AF0000024002098250020303B000830B4074B2C
:100B00001A78074B53F822402368DD69054B0A46E3
:100B1000AC460146204630BC604700BF9825002007
:100B2000303B0008A086010070B501F069FD094C5A
:100B3000094E2070002530682378834208D901F0DF
:100B400059FD336805440133B5F5804F3360F2D366
:100B500070BD00BF992500205825002001F006BE79
:100B600000F1006000F580400068704700F100600F
:100B7000920000F5804001F091BD0000054B1A681D
:100B8000054B1B789B1A834202D9104401F032BDF9
:100B900000207047582500209925002038B5074DC2
:100BA00004462868204401F02DFD28B92868204417
:100BB000BDE8384001F03EBD38BD00BF58250020DB
:100BC00010F0030308D1B0F5007F05D800F1005004
:100BD000A0F508400068704700207047014BC058DE
:100BE000704700BF107AFF1F064991F8243033B1D7
:100BF00000230822086A81F82430FFF7B7BF0120DC
:100C0000704700BF5C250020014B1868704700BF8B
:100C1000002004E070B52A4B1C68C4F30B03240CBD
:100C200063B140F21342934231D040F219429342F1
:100C30002FD040F2214293422DD10323214A0C258B
:100C400005FB03235D6893F9082042F201039C42EF
:100C500024D0B4F5805F23D041F201039C4221D01F
:100C600041F203039C421FD041F207039C4208BF9C
:100C70003122441E0C44013D0B46A3421ED215F9FD
:100C8000016F581C96B1034600F8016CF5E701238B
:100C9000D4E70223D2E73F220B4DD6E73322E3E726
:100CA0004122E1E75A22E4E75922E2E72C25844277
:100CB0001D7001D9981C5A70401A70BD1846FBE788
:100CC000002004E0003B0008E03A0008124B5A887C
:100CD00042F201018A4293B214D0B3F5805F13D07F
:100CE00041F20102934211D041F2030293420FD02C
:100CF00041F2070293420DD10423084A02EB830319
:100D0000D87870470023F8E70123F6E70223F4E7D9
:100D10000323F2E700207047002004E0EC3A0008CB
:100D2000022803D10822034B9A6170470128FCD1A5
:100D30000422F8E700100240022804D14FF40022F8
:100D4000034B9A6170470128FCD14FF48022F7E7EA
:100D500000100240022805D1064A536983F00803B7
:100D6000536170470128FCD1024A536983F00403A0
:100D7000F6E700BF0010024010B50023934203D0F5
:100D8000CC5CC4540133F9E710BD000030B5441EFB
:100D900014F9010F0B4660B193F90050854201F13F
:100DA000010106D11AB993F90020801A30BD013A29
:100DB000EEE7002AF7D1104630BD00000246034698
:100DC000981A13F9011B0029FAD17047024403460F
:100DD000934202D003F8011BFAE770472DE9F04770
:100DE000234C94F8243005468846174683BB2E468C
:100DF000DFF87C90C7B394F824302BB92022FF2170
:100E000048462662FFF7E2FF94F82400C0F1080587
:100E1000BD4228BF3D465FFA85FAAD0041462A46ED
:100E200004EB8000FFF7A8FF94F82430A7EB0A0733
:100E30009A445FFA8AFABAF1080F2E44A844FFB226
:100E400084F824A0D6D1FFF7CFFE0028D2D108E045
:100E5000266A06EB8306B042CAD0FFF7C5FE00281B
:100E6000C5D10020BDE8F0870120BDE8F08700BFB4
:100E70005C250020024B1A78024B1A70704700BFA5
:100E8000982500200024002038B5134C134D20462F
:100E900000F024FC2946204600F04CFC2D68104848
:100EA0006A6D936B23F40023936301F05FF90D499E
:100EB000284600F04BFD6A6D0B48936B0B4943F4D9
:100EC00000239363A0424FF4E1330B6003D0BDE8ED
:100ED000384000F061BB38BDC02C0020383C000811
:100EE00040420F00603C00081C26002084250020A2
:100EF00038B50B4B1A780B4B53F822400A4B9C42E7
:100F000005460CD0094B002118461422FFF75EFF5E
:100F1000056001462046BDE8384000F03DBB38BDC5
:100F200098250020303B0008C02C0020842500209C
:100F3000FEE7000000B59BB0EFF309816822684628
:100F4000FFF71AFFEFF30583034B9A6B9A6A9A6ACD
:100F50009A6A9A6A9B6AFEE700ED00E000B59BB0D2
:100F6000EFF3098168226846FFF706FFEFF3058378
:100F7000044B9A6B9A6A9A6A9A6A9A6A9A6A9B6A04
:100F8000FEE700BF00ED00E000B59BB0EFF3098184
:100F900068226846FFF7F0FEEFF30583034B5A6BB8
:100FA0009A6A9A6A9A6A9A6A9B6AFEE700ED00E07A
:100FB00030B5084D0A4491420BD011F8013B092489
:100FC0005840013CF7D040F300032B4083EA500027
:100FD000F7E730BD2083B8ED002304491A465A5084
:100FE000C8180833802B4260F9D170479C25002037
:100FF000024AD36843F0C003D360704700500040FA
:10100000044B5A6810439A6858600AB1181D10477B
:10101000704700BF1C2600202DE9F0413D4ED6F858
:101020005C54EF682B68DA059CB20CD5202383F35F
:1010300011884FF40070FFF7E3FF6FF480732B60AB
:10104000002383F31188202383F31188DFF8C48001
:1010500014F02F0331D183F31188380613D52106FC
:1010600011D5202383F311882B4800F0F3F90028D1
:1010700044DA0820FFF7C4FF4FF67F733B40EB6074
:10108000002383F311887A060DD563060BD5202340
:1010900083F31188F26C336D9A4201D1336C7BBBC0
:1010A000002383F31188D6F86424D3680BB1106948
:1010B0009847BDE8F04101F0E5BB230712D014F0DA
:1010C000080F0CBF00208020E10748BF40F020003F
:1010D000A20748BF40F04000630748BF40F480705B
:1010E000FFF78EFFA4066B6805D596F8601440469E
:1010F000194000F05FFA2C68A4B2A9E76860BFE766
:1011000027F040073F0410203F0CFFF779FFEF6006
:10111000C6E700BF1C2600205426002010B5054C51
:10112000054A0021204600F015FA044BC4F85C344F
:1011300010BD00BF1C260020F10F00080050004029
:1011400038B5294C037C002918BF0C46012B0546F5
:10115000C0F8644410D1254B98420DD1244B1A6C31
:1011600042F480121A641A6E42F480121A660B213D
:1011700035201B6E00F046F81E4BD5F85C249A42D1
:10118000236802D01C498A422BD11C4901EB530130
:10119000B1FBF3F3A188080442BF23F0070003F07A
:1011A000070343EA40039360E38843F040039BB2A4
:1011B0001361238943F001039BB2536141F404534B
:1011C00043F02C03D36001F4A05100231360B1F568
:1011D000806F136853680CBF7F23FF2385F860344A
:1011E00038BD0749D2E700BF583B00081C26002045
:1011F00000380240001001400014014000BD01050C
:1012000080DE800200F1604300F01F02400903F518
:10121000614309018000C9B200F1604083F8001306
:1012200000F5614001239340C0F8803103607047AE
:10123000F8B5154682680669AA420B46816938BF2F
:101240008568761AB542044607D218462A46FFF743
:1012500093FDA3692B44A3610DE011D932461846D2
:10126000FFF78AFDAF1B3A46E1683044FFF784FD83
:10127000E2683A44A261A3685B1BA3602846F8BDFC
:1012800018462A46FFF778FDE368E4E783682DE90E
:10129000F041044693421546266938BF8568406987
:1012A000361AB5420F4606D22A46FFF765FD636936
:1012B0002B4463610DE012D93246A5EB0608FFF717
:1012C0005BFD4246B919E068FFF756FDE26842440B
:1012D0006261A3685B1BA3602846BDE8F0812A46D3
:1012E000FFF74AFDE368E4E710B50A440024C36150
:1012F000029B006040608460C16081614161026165
:10130000036210BD08B582694369934201D18268C6
:1013100082B98268013282605A1C42611970426946
:1013200003699A4201D3C3684361002100F03AFF88
:10133000002008BD4FF0FF3008BD000070B520232D
:1013400004460E4683F31188A568A5B1A368A26977
:10135000013BA360531CA36115782269934224BF0B
:10136000E368A361E3690BB120469847002383F348
:101370001188284670BD3146204600F003FF002842
:10138000E2DA85F3118870BD2DE9F74F05460F4667
:1013900090469A46D0F81C90202686F311884FF08C
:1013A000000B144664B1224639462846FFF740FF39
:1013B000034668B95146284600F0E4FE0028F1D003
:1013C000002383F31188A8EB040003B0BDE8F08F7D
:1013D000B9F1000F03D001902846C847019B8BF359
:1013E0001188E41A1F4486F31188DBE7C16081612C
:1013F0004161C3611144009B0060406082600161F3
:1014000003627047F8B504460E461746202383F35F
:101410001188A568A5B1A368013BA36063695A1C44
:1014200062611E70236962699A4224BFE368636146
:10143000E3690BB120469847002080F31188F8BD7E
:101440003946204600F09EFE0028E2DA85F3118836
:10145000F8BD0000836942699A4210B501D18268E3
:101460007AB98268013282605A1C82611C780369F1
:101470009A4201D3C3688361002100F093FE2046A5
:1014800010BD4FF0FF3010BD2DE9F74F05460F4658
:1014900090469A46D0F81C90202686F311884FF08B
:1014A000000B144664B1224639462846FFF7EEFE8B
:1014B000034668B95146284600F064FE0028F1D082
:1014C000002383F31188A8EB040003B0BDE8F08F7C
:1014D000B9F1000F03D001902846C847019B8BF358
:1014E0001188E41A1F4486F31188DBE70268436819
:1014F0001143016003B11847704700001430FFF733
:1015000043BF00004FF0FF331430FFF73DBF000032
:101510003830FFF7B9BF00004FF0FF333830FFF726
:10152000B3BF00001430FFF709BF00004FF0FF31D8
:101530001430FFF703BF00003830FFF763BF00002F
:101540004FF0FF323830FFF75DBF000000207047DA
:10155000FFF7E4BD37B50F4B0360002343608360A2
:10156000C360012304460374154600900B464FF4F4
:10157000007200F15C011430FFF7B6FE00942B46B8
:101580004FF4007204F5177104F13800FFF72EFFD5
:1015900003B030BD6C3B000810B52023044683F334
:1015A0001188FFF7CDFD02232374002383F31188F4
:1015B00010BD000038B5C36904460D461BB90421AF
:1015C0000844FFF793FF294604F11400FFF79AFE41
:1015D000002806DA201D4FF48061BDE83840FFF78F
:1015E00085BF38BD026843681143016003B11847E5
:1015F0007047000013B5446BD4F894341A6811781E
:10160000042915D1217C022912D1197912890123CB
:101610008B4013420CD101A904F14C0001F0E8FE0B
:10162000D4F89444019B21790246206800F0DAF94D
:1016300002B010BD143001F06BBE00004FF0FF335C
:10164000143001F065BE00004C3001F03DBF0000D9
:101650004FF0FF334C3001F037BF0000143001F081
:1016600039BE00004FF0FF31143001F033BE0000EE
:101670004C3001F009BF00004FF0FF324C3001F058
:1016800003BF0000D0F8942438B5136819780429F2
:10169000054601D0012038BD017C0229FAD112791A
:1016A0005C89012090400440F4D105F1140001F060
:1016B000CBFD02460028EDD0D5F894544FF480734A
:1016C0002868697900F07CF9204638BD406BFFF747
:1016D000D9BF000000207047704700007FB5124B53
:1016E0000360002343608360C360012502260F4B23
:1016F000057404460290019300F184022946009685
:101700004FF48073143001F07BFD094B0193029478
:1017100000964FF4807304F52372294604F14C00BF
:1017200001F042FE04B070BD943B0008CD160008E5
:10173000F51500080B68202282F311880A7903EB63
:10174000820290614A79093243F822008A7912B103
:1017500003EB8203986102230374C0F894140023FE
:1017600083F311887047000038B5037F044613B136
:1017700090F85430ABB9201D01250221FFF732FF4C
:1017800004F1140025776FF0010100F017FD84F8D3
:10179000545004F14C006FF00101BDE8384000F0F6
:1017A0000DBD38BD10B5012104460430FFF71AFF06
:1017B0000023237784F8543010BD000038B5044668
:1017C0000025143001F034FD04F14C00257701F0C0
:1017D00003FE201D84F854500121FFF703FF20462B
:1017E000BDE83840FFF74EBF90F8443003F0600387
:1017F000202B19D190F84520212A0AD0222A4FF017
:1018000000030ED0202A0FD1084A82630722C26348
:1018100004E0064B83630723C363002303640120B2
:1018200070478363C363F9E70020704701240020F9
:10183000D0F8943437B51A681178042904461AD1BF
:10184000017C022917D11979128901238B40134297
:1018500011D100F14C05284601F07EFE58B101A9D6
:10186000284601F0C5FDD4F89444019B2179024635
:10187000206800F0B7F803B030BD000000EB810332
:10188000F7B59C6905460E46F4B1202383F3118811
:1018900005EB8607201D0821FFF7A4FEFB685B69A6
:1018A0001B684C3413B1204601F0B0FD01A920465D
:1018B00001F09EFD024648B1019B3146284600F0EA
:1018C00091F8002383F3118803B0F0BDFB685A69D7
:1018D0001268002AF5D01B8A013B1340F1D105F1B3
:1018E0004402EAE7093138B550F82140DCB1202341
:1018F00083F31188D4F894241368527903EB82039C
:10190000DB689B695D6845B104216018FFF76AFEDA
:10191000294604F1140001F0A1FC2046FFF7B2FEB5
:10192000002383F3118838BD7047000001F062B8CE
:101930000123037000234360C36183620362C362B7
:1019400043620363038143817047000038B5044656
:10195000202383F3118800254160C560056145613E
:10196000856101F057F80223237085F3118838BD93
:1019700070B500EB810305465069DA600E461446E7
:1019800018B110220021FFF721FAA06918B1102226
:101990000021FFF71BFA31462846BDE8704001F0F0
:1019A00003B90000028902F001020281428902F0BB
:1019B00001024281002202614261826101F088B924
:1019C000F0B400EB81044789E4680125A4698D40E7
:1019D0003D43458123600023A2606360F0BC01F0B9
:1019E000A3B90000F0B400EB81040789E468012585
:1019F00064698D403D43058123600023A2606360DC
:101A0000F0BC01F01DBA000070B5022300250446A9
:101A10000370A0F84C5080F84E5080F84F5005816C
:101A20004581C56005614561856180F8345001F0EC
:101A300057F863681B6823B129462046BDE870400B
:101A4000184770BD436802781B6880F85020052253
:101A500002700BB10421184770470000436890F8EA
:101A600050201B6802700BB1052118477047000019
:101A700090F8343070B5044613B1002380F8343048
:101A800004F14402204601F045F963689B6863BB9A
:101A900094F8445015F0600615D194F8453005F0DF
:101AA0007F0545EA032540F202339D4200F00E8196
:101AB0005BD8022D00F0DC803FD8002D00F087803D
:101AC000012D00F0CF800021204601F07BFB00219A
:101AD000204601F06DFB63681B6813B106212046A8
:101AE0009847062384F8343070BD20469847002874
:101AF000CED094F84B2094F84A3043EA0223E26BAC
:101B0000934238BFE36394F94430E56B002B4FF008
:101B1000200380F2FD80002D00F0EC80092284F883
:101B2000342083F311880021E36BA26B2046FFF77A
:101B300059FF002383F3118870BDB5F5817F00F054
:101B4000B180B5F5407F49D0B5F5807FBBD194F821
:101B50004630012BB7D1B4F84C3023F00203A4F87F
:101B60004C30A663E6632664C3E740F201639D42FE
:101B70001ED8B5F5C06F3BD2B5F5A06FA3D1B4F8B0
:101B80004430B3F5A06F0ED194F8463084F84E304F
:101B9000204600F0FDFF63681B6813B10121204659
:101BA0009847032323700023A363E3632364A0E720
:101BB000B5F5106F32D040F602439D4252D0B5F5D4
:101BC000006F80D104F14F03A363012324E004F1EB
:101BD0004C03A3630223E36325648AE794F8463049
:101BE000012B7FF470AFB4F84C3043F00203B6E73A
:101BF00094F84920616894F848304D6894F847108B
:101C000043EA0223204694F84620A84700283FF4E0
:101C10005AAF4368A3630368E363A4E72378042B04
:101C200010D1202383F311882046FFF7BBFE86F3F3
:101C30001188636884F84F601B68032121700BB121
:101C40002046984794F84630002BACD084F84F30AB
:101C50000423237063681B68002BA4D00221204654
:101C60009847A0E7374BA3630223E36300239DE774
:101C700094F8481011F0800F204601F00F010ED0AB
:101C800001F03AF8012806D002287FF41CAF2E4B51
:101C9000A363E06367E72D4BA363E56363E701F0AC
:101CA0001DF8EFE794F84630002B7FF40CAF94F862
:101CB000483013F00F013FF476AF1A06204602D5E4
:101CC00001F094FA6FE701F087FA6CE794F8463078
:101CD000002B7FF4F8AE94F8483013F00F013FF476
:101CE00062AF1B06204602D501F06CFA5BE701F0FB
:101CF0005FFA58E7142284F8342083F311882B46C6
:101D00002A4629462046FFF75BFE85F3118870BD01
:101D10005DB1152284F8342083F311880021E36B30
:101D2000A26B2046FFF74CFE03E70B2284F8342019
:101D300083F311882B462A4629462046FFF752FE98
:101D4000E3E700BFC43B0008BC3B0008C03B000801
:101D500038B590F834300446152B29D8DFE803F065
:101D60003E28282828283E28280B293928282828D2
:101D7000282828283E3E90F84B1090F84A20C36B44
:101D800042EA01229A4214D9C268128AB3FBF2F5E0
:101D900002FB15356DB9202383F311882B462A46A3
:101DA0002946FFF71FFE85F311880A2384F8343093
:101DB00038BD142384F83430202383F311880023A2
:101DC0001A4619462046FFF7FBFD002383F31188CE
:101DD00038BD036C03B198470023E7E7002101F009
:101DE000F1F90021204601F0E3F963681B6813B1A3
:101DF0000621204698470623D8E7000090F83420B3
:101E0000152A38B5044622D80123934040F6416292
:101E100013421DD113F480150FD19B0217D50B234C
:101E200080F83430202383F311882B462A46294634
:101E3000FFF7D8FD85F3118838BDC3689B695B68DF
:101E40002BB9036C03B19847002384F8343038BDB4
:101E5000002101F0B7F90021204601F0A9F96368DB
:101E60001B6813B10621204698470623EDE70000C2
:101E7000024B00221B605B609A607047842A00203E
:101E8000002303748268054B1B6899689142FBD25A
:101E90005A6803604260106058607047842A0020CE
:101EA00008B5202383F31188037C032B05D0042B72
:101EB0000DD02BB983F3118808BD436900221A6045
:101EC0004FF0FF334361FFF7DBFF0023F2E790E8B9
:101ED0000C001A6002685360F2E7000000230374EC
:101EE0008268054B1B6899689142FBD85A68036069
:101EF0004260106058607047842A0020054B1969C1
:101F00000874186802681A6053601861012303742A
:101F1000FEF7FAB9842A002030B54B1C87B005467D
:101F20000A4C10D023690A4A01A800F063F9284638
:101F3000FFF7E4FF049B13B101A800F097F92369B0
:101F4000586907B030BDFFF7D9FFF8E7842A0020B1
:101F5000A11E000838B50C4D41612B6981689A6853
:101F60009142044603D8BDE83840FFF789BF1846C0
:101F7000FFF786FF01232C61014623742046BDE84C
:101F80003840FEF7C1B900BF842A0020044B1A680C
:101F90001B6990689B68984294BF0020012070479D
:101FA000842A002010B5084C236820691A68226032
:101FB0005460012223611A74FFF790FF01462069E3
:101FC000BDE81040FEF7A0B9842A0020FEE700001B
:101FD00010B5174CFFF74CFF00F0FEF880221549B2
:101FE000204600F083F8012344F8180C0374124BC8
:101FF000124AD96821F4E0610904090C0A43104926
:10200000DA60CA6842F08072CA600E490A6842F01B
:1020100001020A601022DA77202283F822200023AE
:1020200083F3118862B60848BDE8104000F080B81C
:10203000AC2A0020C83B000800ED00E00003FA05D0
:10204000F0ED00E0001000E0D03B00082DE9F84F73
:102050001F4CDFF88090656904F114074FF0000809
:10206000D9F82430266AAA689E1B96421DD34FF0E9
:10207000200AAA68236AD5F80CB0134423622B689F
:10208000BB425F60A6EB02066361C5F80C8001D11C
:1020900001F08EFA88F311882869D8478AF31188ED
:1020A0006569AB689E42E4D2DAE76269BA420CD055
:1020B000916823628E1B9660A86802282CBF1818AE
:1020C000981CBDE8F84F01F079BABDE8F88F00BF61
:1020D000842A0020000C0040034B59685A68521AA9
:1020E0009042FBD8704700BF001000E082600222DF
:1020F00002740022427470478368A3F17C0243F8A3
:102100000C2C026943F83C2C426943F8382C074AEE
:1021100043F81C2CC26843F8102C022203F8082C48
:10212000002203F8072CA3F11800704721030008D0
:1021300010B5202383F31188FFF7DEFF002104464A
:10214000FFF708FF002383F31188204610BD00002D
:10215000024B1B6958610F20FFF7D0BE842A002074
:10216000202383F31188FFF7F3BF000008B5014671
:10217000202383F311880820FFF7CEFE002383F38A
:10218000118808BD49B1064B42681B6918605A6046
:10219000136043600420FFF7BFBE4FF0FF3070476D
:1021A000842A00200368984206D01A6802605060B2
:1021B00059611846FFF764BE7047000038B5044601
:1021C0000D462068844200D138BD036823605C60FE
:1021D0004561FFF755FEF4E7054B03F114025A6120
:1021E0009A614FF0FF32DA6100221A62704700BF35
:1021F000842A0020F8B503611A4BC2605C6A1A4B4E
:102200001A46022952F8145F38BF02219542064649
:102210001F460AD1586198611C6205604560816063
:102220000819BDE8F84001F0B9B9186AAB68241A7A
:102230000C1902D3E41A2D6804E09C4202D2204417
:1022400001F0BCF9AB689C42F4D86B6873603560F0
:102250001E606E60B460A9684FF0FF33091BA9606F
:10226000FB61F8BD000C0040842A002010B41A4C19
:10227000234653F8141F814210D0416802680A6057
:10228000026851609A424FF00001C16003D0936828
:1022900081680B4493605DF8044B70470A68626183
:1022A00000209A425360C86003D15DF8044B01F0EE
:1022B0007FB99368886803449360084A206A526A29
:1022C000121A9342E7D9991A012998BF931C18440E
:1022D0005DF8044B01F072B9842A0020000C004024
:1022E00000207047FEE70000704700004FF0FF300D
:1022F00070470000022906D0032906D001290648AC
:1023000018BF0020704705487047032A9ABF044849
:1023100000EBC20000207047BC3C0008703C000885
:102320000824002070B59AB001AD0646084629463B
:10233000144600F095F82846FEF740FDC0B2431C55
:102340005B0086E8180023700323637000230234C7
:102350001946DAB2904204F1020401D81AB070BDF5
:10236000EA5C04F8022C04F8011C0133F1E70000D8
:1023700008B5202383F311880348FFF759FA002397
:1023800083F3118808BD00BFC02C002010B504469F
:10239000052916D8DFE801F016150316161D2023AF
:1023A00083F311880E4A0121FFF7E2FA20460D4A15
:1023B0000221FFF7DDFA0C48FFF700FA002383F350
:1023C000118810BD202383F311880748FFF7CCF94B
:1023D000F4E7202383F311880348FFF7E3F9EDE7DF
:1023E000F03B0008143C0008C02C002038B50C4D10
:1023F0000C4C0D492A4604F10800FFF793FF05F144
:10240000CA0204F110000949FFF78CFF05F5CA72F2
:1024100004F118000649BDE83840FFF783BF00BF4C
:102420008831002008240020403C00084A3C000875
:10243000553C000870B5044608460D46FEF7BEFC44
:10244000C6B22046013403780BB9184670BD324637
:102450002946FEF79BFC0028F3D1012070BD000047
:102460002DE9F04704460D46FEF7A8FC2B49C6B2FD
:102470002046FFF7DFFF08B10936F6B228492046AB
:10248000FFF7D8FF08B11036F6B2632E0BD8DFF88D
:102490008C80DFF88C90234FDFF894A0267846B923
:1024A0002E70BDE8F08721462846BDE8F04701F0D0
:1024B0000BBB252E2DD1072241462046FEF766FC98
:1024C00060B9194B2A4603F1100153F8040B42F886
:1024D000040B8B42F9D107341035DFE70822494657
:1024E0002046FEF753FCA0B9104BAA1C13F8011F9D
:1024F00009095345C95D02F8021C197801F00F0162
:1025000002F10202C95D02F8031CEFD1183508344C
:10251000C4E72E7001340135C0E700BFDC3C000881
:10252000553C0008F53C0008E43C00080F7AFF1F0A
:102530001B7AFF1FBFF34F8F024AD368DB03FCD423
:10254000704700BF003C024008B5094B1B7873B9C7
:10255000FFF7F0FF074B1A69002ABFBF064A5A600F
:1025600002F188325A601A6822F480621A6008BD4B
:10257000E6330020003C02402301674508B50B4BC1
:102580001B7893B9FFF7D6FF094B1A6942F0004256
:102590001A611A6842F480521A601A6822F4805252
:1025A0001A601A6842F480621A6008BDE63300209F
:1025B000003C0240172870B513D80B4A0B4C137817
:1025C00063B90B4E4FF0006144F8231056F82350C6
:1025D0000133182B2944F7D10123137054F820003C
:1025E00070BD002070BD00BF48340020E8330020DB
:1025F000083D0008014B53F820007047083D0008D3
:1026000018207047172810B5044601D9002010BDC6
:10261000FFF7D0FF064B53F824301844C21A0BB909
:10262000012010BD12680132F0D1043BF6E700BF73
:10263000083D0008172810B5044629D8FFF77AFF8F
:10264000FFF782FF1349F323CB600C23B0FBF3F2B7
:1026500003FB1200D30143EAC003DBB243F400736F
:1026600043F002030B610B6943F480330B61FFF706
:1026700061FF2046FFF79EFF074B53F8241000F040
:10268000DDF8FFF77BFF2046BDE81040FFF7BABF3B
:10269000002010BD003C0240083D00082DE9F84331
:1026A00012F00103154640D18218B2F1026F3CD2FC
:1026B0002C4B1B6813F0010337D02B4CFFF744FF62
:1026C000F323E360FFF736FF40F20127032D01D922
:1026D000830713D0244C0F46401A40F20118EB1B1D
:1026E0000B44012B00EB0706236924D823F00103D8
:1026F0002361FFF743FF0120BDE8F883236923F43A
:102700004073236123693B43236151F8046B0660E6
:10271000BFF34F8FFFF70EFF03689E4208D0236977
:1027200023F001032361FFF729FF0020BDE8F883B0
:10273000043D0430CAE723F440732361236943EA6C
:1027400008032361B94637F8023B3380BFF34F8F4C
:10275000FFF7F0FE3688B9F80030B6B2B342BED00B
:10276000DDE700BF00380240003C0240084908B5E0
:102770000B7828B153B9FFF7E7FE01230B7008BDB2
:1027800023B1BDE808400870FFF7F8BE08BD00BFE0
:10279000E633002010B50244064B0439D2B2904211
:1027A00000D110BD441C00B253F8200041F8040FC2
:1027B000E0B2F4E750280040104B30B51C6F240401
:1027C00007D41C6F44F400741C671C6F44F400446D
:1027D0001C670B4C236843F4807323600244094B4D
:1027E0000439D2B2904200D130BD441C00B251F83D
:1027F000045F43F82050E0B2F4E700BF0038024025
:10280000007000405028004007B5012201A90020B7
:10281000FFF7C0FF019803B05DF804FB13B5044651
:10282000FFF7F2FFA04206D002A9012241F8044DB1
:102830000020FFF7C1FF02B010BD0000704700008C
:10284000034B1B689B0042BF024B01221A7070476A
:102850007438024049340020014B1878704700BF9B
:1028600049340020064A536823F001035360EFF314
:102870000983683383F30988002383F31188704741
:1028800030EF00E010B5202383F31188104B5B6814
:1028900013F4006318D0F1EE103AEFF309844FF00F
:1028A000807344F84C3C0B4BDB6844F8083CA4F1C3
:1028B000680383F30988FFF769FB18B1064B44F8F6
:1028C000503C10BD054BFAE783F3118810BD00BFE3
:1028D00000ED00E030EF00E03103000834030008B1
:1028E00070470000FEE70000084A094B09498B4287
:1028F00004D3094A0021934205D3704752F8040FCC
:1029000043F8040BF3E743F8041BF4E7BC3E00086C
:10291000C4340020C4340020C4340020836D30B59A
:1029200000229D68446D11464FF0FF3004EB4213C6
:1029300001329542C3F80019C3F81019C3F8080909
:10294000C3F8001BC3F8101BC3F8080BEED24FF0FE
:102950000113C4F81C3830BD890141F02001016128
:1029600003699B06FCD41220FFF7B6BB204B03EB98
:1029700080022DE9F047D2F80CE05D6DDEF81420FE
:10298000461CD2F800C005EB063605EB401851682E
:1029900061450BD3D5F83428012303FA00F022EA6D
:1029A0000000C5F834081846BDE8F087BEF81040AE
:1029B000ACEB0103A34228BF2346D8F81849A4B2C0
:1029C000B3EB840F10D894681F46A4F1040959F89A
:1029D00004AFC6F800A0042F01D9043FF7E71C4458
:1029E0000B4494605360D2E70020BDE8F08700BF3D
:1029F0004C34002010B5054C2046FEF799FF4FF0EF
:102A0000A0436365024BA36510BD00BF4C3400209A
:102A10008C3D00080378012B70B5054650D12A4B38
:102A2000446D98421BD1294B5A6B42F080025A6385
:102A30005A6D42F080025A655A6D5A6942F080021E
:102A40005A615A6922F080025A610E2143205B6963
:102A5000FEF7D8FB1E4BE3601E4BC4F80038002382
:102A6000C4F8003EC02323606E6D4FF45023A3636F
:102A70003369002BFCDA012333610C20FFF72CFBB8
:102A80003369DB07FCD41220FFF726FB3369002BE8
:102A9000FCDA0026A6602846FFF740FF6B68C4F802
:102AA0001068DB68C4F81468C4F81C684BB90A4B9A
:102AB000A3614FF0FF336361A36843F00103A36098
:102AC00070BD064BF4E700BF4C34002000380240D4
:102AD0004014004003002002003C30C0083C30C0DD
:102AE000F8B5446D054600212046FFF735FFA96D76
:102AF00000234FF001128F68C4F834384FF000669D
:102B0000C4F81C284FF0FF3004EB431201339F42FE
:102B1000C2F80069C2F8006BC2F80809C2F8080BD5
:102B2000F2D20B686A6DEB6563621023136116695C
:102B300016F01006FBD11220FFF7CEFAD4F80038B9
:102B400023F4FE63C4F80038A36943F4402343F040
:102B50001003A3610923C4F81038C4F814380A4BD1
:102B6000EB604FF0C043C4F8103B084BC4F8003B87
:102B7000C4F81069C4F80039EB6D03F1100243F496
:102B80008013EA65A362F8BD683D0008408000102C
:102B9000426D90F84E10D2F8003823F4FE6343EAF9
:102BA0000113C2F8003870472DE9F0410EB200EB76
:102BB00086080D46D8F80C100F6807F00303022BA7
:102BC00050D0032B50D03D4A3D4F012B18BF174624
:102BD000446D4FEA451E04EB0E030022C3F8102B90
:102BE0008A6905F1100C002A40D04A8A05F1580381
:102BF0005B013A43E2500123D4F81C2803FA0CF39A
:102C00001343A6444A69C4F81C380023CEF810398F
:102C100005F13F03002A39D00A8A898B92080129DD
:102C200088BF4A43C16D04EB8303561841EA024250
:102C3000C66529465A602046FFF78EFED8F80C304C
:102C40001B8A43EA85531F4305F148035B01E750A4
:102C50000123D4F81C2803FA05F51543C4F81C58C1
:102C6000BDE8F081174FB3E7174FB1E704EB461308
:102C7000D3F8002B22F40042C3F8002BD4F81C2810
:102C8000012303FA0CF322EA0303BAE704EB8303FC
:102C90000E4A5A6004EB461629462046FFF75CFEB2
:102CA000D6F8003923F40043C6F80039D4F81C38AC
:102CB000012202FA05F523EA0505CFE7008000109E
:102CC000008004100080081000800C100004000236
:102CD000826D1268C265FFF721BE00005831436D56
:102CE00049015B5813F4004004D013F4001F14BFD3
:102CF00001200220704700004831436D49015B58B4
:102D000013F4004004D013F4001F14BF012002206C
:102D10007047000000EB8101CB68196A0B681360F3
:102D20004B6853607047000000EB810330B5DD68ED
:102D3000AA691368D36019B9402B84BF402313607C
:102D40006B8A1468426D1C44013CB4FBF3F463438A
:102D5000033323F0030302EB411043EAC44343F07F
:102D6000C043C0F8103B2B6803F00303012B09B2EA
:102D70000ED1D2F8083802EB411013F4807FD0F85E
:102D8000003B14BF43F0805343F00053C0F8003BB6
:102D900002EB4112D2F8003B43F00443C2F8003B7F
:102DA00030BD00002DE9F041244D6E6D06EB40135F
:102DB0000446D3F8087BC3F8087B38070AD5D6F851
:102DC0001438190706D505EB84032146DB6828462D
:102DD0005B689847FA072FD5D6F81438DB072BD550
:102DE00005EB8403D968CCB98B69488A5E68B6FB69
:102DF000F0F200FB12628AB91868DA6890420DD2CC
:102E0000121A83E81400202383F311880B4821460B
:102E1000FFF78AFF84F31188BDE8F081012303FAEC
:102E200004F26B8923EA02036B81CB6823B121464C
:102E30000248BDE8F0411847BDE8F0814C3400205D
:102E400000EB810370B5DD68436D6C692668E66050
:102E50004A0156BB1A444FF40020C2F810092A68F0
:102E600002F00302012A0AB20ED1D3F8080803EBDC
:102E7000421410F4807FD4F8000914BF40F0805051
:102E800040F00050C4F8000903EB4212D2F80009E8
:102E900040F00440C2F80009D3F83408012202FAD5
:102EA00001F10143C3F8341870BD19B9402E84BF35
:102EB0004020206020682E8A841940F00050013C98
:102EC0001A44B4FBF6F440EAC440C6E7F8B5044639
:102ED0001E48456D05EB4413D3F80869C3F808692B
:102EE000F10717D5D5F81038DA0713D500EB8403AE
:102EF000D9684B691F68DA68974218D2D21B00273D
:102F00001A605F60202383F311882146FFF798FF42
:102F100087F31188330617D5D5F834280123A34049
:102F2000134211D02046BDE8F840FFF71FBD012332
:102F300003FA04F2038923EA020303818B68002B5E
:102F4000E8D021469847E5E7F8BD00BF4C340020A3
:102F500096482DE9F84F456D6E69AB691E4016F431
:102F6000805F6E61044605D0FEF74EFDBDE8F84F68
:102F7000FFF788BC002E12DAD5F8003E8B489B077D
:102F80001EBFD5F8003E23F00303C5F8003ED5F878
:102F9000043823F00103C5F80438FEF75FFD370558
:102FA00002D58248FEF74EFDB0040CD5D5F808389E
:102FB00013F0060FEB6823F470530CBF43F4105367
:102FC00043F4A053EB60310704D56368DB680BB1B1
:102FD00076489847F2025AD4B3020CD5D4F85480FC
:102FE000DFF8C8A100274FF00109A36D9B68F9B273
:102FF0008B4280F08780F70619D5616D0A6AC2F3AB
:103000000A1702F00F0302F4F012B2F5802F00F05D
:10301000A180B2F5402F0AD104EB830301F5805162
:10302000DB68186A00231A469F4240F0878030030D
:10303000D5F8184813D5E10302D50020FFF7B2FEFA
:10304000A20302D50120FFF7ADFE630302D50220E3
:10305000FFF7A8FE270302D50320FFF7A3FE7503A1
:1030600084D5E00702D50020FFF730FFA10702D585
:103070000120FFF72BFF620702D50220FFF726FF92
:1030800023077FF573AF0320FFF720FF6EE7D4F827
:103090005480DFF818A100274FF00109A36D9B6849
:1030A0005FFA87FB5B4597D308EB4B13D3F80029F6
:1030B00002F44022B2F5802F22D1D3F80029002A51
:1030C0001EDAD3F8002942F09042C3F80029D3F861
:1030D0000029002AFBDB5946606DFFF73DFC228981
:1030E00009FA0BF322EA0303238104EB8B03DB6869
:1030F0009B6813B15946504698475846FFF736FC2F
:103100000137CBE708EB4112D2F8003B03F4402330
:10311000B3F5802F10D1D2F8003B002B0CDA628976
:1031200009FA01F322EA0303638104EB8103DB68FC
:10313000DB680BB150469847013756E79C0708BF3C
:103140000A68072B98BF027003F101039CBF120AA3
:10315000013069E7023304EB830201F580515268C4
:1031600090690268D0F808C04068A2EB000E002207
:10317000104697420AD104EB830463689B699A68FE
:103180003A449A605A6817445F6050E712F0030FA0
:1031900008BF0868964588BF8CF8000002F101025C
:1031A00084BF000A0CF1010CE3E700BF4C3400209F
:1031B000436D03EB4111D1F8003B43F40013C1F818
:1031C000003B7047436D03EB4111D1F8003943F4E4
:1031D0000013C1F800397047436D03EB4111D1F87A
:1031E000003B23F40013C1F8003B7047436D03EB31
:1031F0004111D1F8003923F40013C1F800397047A8
:1032000030B5039C0172043304FB0325C361049BA6
:1032100003630021059B00604060C1604261026160
:103220008561046242628162C162436330BD000015
:103230000022416A41610161C2608262C2626FF034
:103240000101FEF7BBBF000003694269934203D14D
:10325000C2680AB100207047181D704703691960E1
:10326000C2680132C260C269134482690361934239
:1032700024BF436A03610021FEF794BF38B50446BA
:103280000D46E3683BB16269131D1268A3621344E3
:10329000E362002038BD237A33B929462046FEF781
:1032A00071FF0028EDDA38BD6FF00100FBE7000088
:1032B000C368C269013BC3604369134482694361C7
:1032C000934224BF436A436100238362036B03B1CB
:1032D0001847704770B52023044683F31188866A27
:1032E0003EB9FFF7CBFF054618B186F31188284693
:1032F00070BDA36AE26A13F8015BA362934202D332
:103300002046FFF7D5FF002383F31188EFE7000085
:103310002DE9F84F04460E4690469946202787F33C
:1033200011880025AA46D4F828B0BBF1000F09D1B6
:1033300049462046FFF7A2FF20B18BF311882846AB
:10334000BDE8F88FA16AE36AA8EB050B5B1A9B4501
:1033500028BF9B46BBF1400F1BD9334601F1400209
:1033600051F8040B43F8040B9142F9D1A36A40339E
:103370004036A3624035A26AE36A9A4202D32046ED
:10338000FFF796FF8AF311884545D8D287F3118855
:10339000C9E730465A46FDF7EFFCA36A5B445E443A
:1033A000A3625D44E7E7000010B5029C017204339C
:1033B00003FB0421C36100238362C362039B036395
:1033C000049B00604060C4604261026181610462EC
:1033D0004262436310BD0000026AC260426A4261F9
:1033E000026100228262C2626FF00101FEF7E6BE56
:1033F000436902699A4203D1C2680AB1002070474A
:10340000184650F8043B0B6070470000C368C2695F
:103410000133C3604369134482694361934224BF0B
:10342000436A43610021FEF7BDBE000038B5044683
:103430000D46E3683BB123691A1DA262E269134499
:10344000E362002038BD237A33B929462046FEF7CF
:1034500099FE0028EDDA38BD6FF00100FBE70000AF
:1034600003691960C268013AC260C2691344826983
:103470000361934224BF436A036100238362036BA9
:1034800003B118477047000070B5202304460E466C
:1034900083F31188856A35B91146FFF7C7FF10B16C
:1034A00085F3118870BDA36A1E70A36AE26A0133B6
:1034B0009342A36204D3E16920460439FFF7D0FFA9
:1034C000002080F3118870BD2DE9F84F04460D46A9
:1034D00091469A464FF0200888F311880026B3469B
:1034E000A76A4FB951462046FFF7A0FF20B187F3E6
:1034F00011883046BDE8F88FA06AE76AA9EB060399
:103500003F1A9F4228BF1F46402F1BD905F1400399
:1035100055F8042B40F8042B9D42F9D1A36A40339F
:10352000A3624036A26AE36A9A4204D3E169204664
:103530000439FFF795FF8BF311884E45D9D288F3F4
:103540001188CDE729463A46FDF716FCA36A3B44AD
:103550003D44A3623E44E5E7026943699A4203D1D0
:10356000C3681BB9184670470023FBE7836A002B2A
:10357000F8D0043B9B1AF5D01360C368013BC360CD
:10358000C3691A44836902619A4224BF436A036192
:10359000002383620123E5E700F0A4B8034B002277
:1035A00058631A610222DA60704700BF000C0040C5
:1035B000014B0022DA607047000C0040014B586359
:1035C000704700BF000C00404B6843608B6883600D
:1035D000CB68C3600B6943614B6903628B694362CB
:1035E0000B6803607047000008B5224B22481A6937
:1035F00040F2FF110A431A611A6922F4FF7222F0A5
:1036000001021A611A691A6B0A431A631A6D0A4396
:103610001A651A4A1B6D1146FFF7D6FF184802F1CA
:103620001C01FFF7D1FF174802F13801FFF7CCFF6B
:10363000154802F15401FFF7C7FF144802F1700169
:10364000FFF7C2FF124802F18C01FFF7BDFF1148DE
:1036500002F1A801FFF7B8FF0F4802F1C401FFF71C
:10366000B3FF0E4802F1E001FFF7AEFFBDE80840EE
:1036700000F0A4B80038024000000240983D000865
:103680000004024000080240000C0240001002400A
:103690000014024000180240001C024000200240BA
:1036A00008B500F0FFF9FEF793FCFFF7C9F8BDE895
:1036B0000840FEF79BBE000070470000084B1A69E7
:1036C000920710B508D500241C61202383F31188CC
:1036D000FEF7BCFC84F31188BDE81040FFF7D2B8B8
:1036E000000C0040104B1A6C42F008021A641A6E6B
:1036F00042F008021A660D4A1B6E936843F00803F5
:1037000093600B4B53229A624FF0FF32DA62002231
:103710009A615A63DA605A6001225A6108211A607C
:103720003220FDF76FBD00BF00380240002004E0EA
:10373000000C00401F4B1A696FEAC2526FEAD25266
:103740001A611A69C2F308021A614FF0FF301A6950
:103750005A69586100215A6959615A691A6A62F0B6
:1037600080521A621A6A02F080521A621A6A5A6AFF
:1037700058625A6A59625A6A1A6C42F080521A6444
:103780001A6E42F080521A661A6E0B4A106840F4A4
:1037900080701060186F00F44070B0F5007F1EBF9D
:1037A0004FF4803018671967536823F4007353602F
:1037B00000F058B90038024000700040324B4FF022
:1037C00080521A64314A4FF4404111601A6842F045
:1037D00001021A601A689207FCD59A6822F0030267
:1037E0009A60294B19469A6812F00C02FBD11868AE
:1037F00000F0F90018609A601A6842F480321A608A
:103800000B689B03FCD54B6F43F001034B671E4BCA
:103810005A6F9007FCD51E4A5A601A6842F08072AF
:103820001A601A4A53685904FCD5174B1A6892015A
:10383000FCD5184A9A600322C3F88C20164B1A68EC
:10384000164B9A42164B1BD1164A1168164A9142E2
:1038500016D140F205121A600B4B9A6842F0020230
:103860009A609A6802F00C02082AFAD15A6C42F463
:1038700080425A645A6E42F480425A665B6E7047C8
:1038800040F20572E7E700BF0038024000700040D8
:103890001854400700948838002004E01164002088
:1038A000003C024000ED00E041C20F41084A08B56B
:1038B000536911680B4003F00103536123B1054ABA
:1038C00013680BB150689847BDE80840FEF7DABFAF
:1038D000003C01409C250020084A08B55369116846
:1038E0000B4003F00203536123B1054A93680BB107
:1038F000D0689847BDE80840FEF7C4BF003C0140CF
:103900009C250020084A08B5536911680B4003F054
:103910000403536123B1054A13690BB150699847F9
:10392000BDE80840FEF7AEBF003C01409C250020EA
:10393000084A08B5536911680B4003F00803536146
:1039400023B1054A93690BB1D0699847BDE8084097
:10395000FEF798BF003C01409C250020084A08B5AE
:10396000536911680B4003F01003536123B1054AFA
:10397000136A0BB1506A9847BDE80840FEF782BF52
:10398000003C01409C250020174B10B55C691A686B
:10399000144004F478725A61A30604D5134A936A5A
:1039A0000BB1D06A9847600604D5104A136B0BB16F
:1039B000506B9847210604D50C4A936B0BB1D06B22
:1039C0009847E20504D5094A136C0BB1506C98472F
:1039D000A30504D5054A936C0BB1D06C9847BDE89C
:1039E0001040FEF74FBF00BF003C01409C25002067
:1039F0001A4B10B55C691A68144004F47C425A6191
:103A0000620504D5164A136D0BB1506D9847230516
:103A100004D5134A936D0BB1D06D9847E00404D5DB
:103A20000F4A136E0BB1506E9847A10404D50C4A8F
:103A3000936E0BB1D06E9847620404D5084A136F99
:103A40000BB1506F9847230404D5054A936F0BB10F
:103A5000D06F9847BDE81040FEF714BF003C01400E
:103A60009C250020062108B50846FDF7CBFB062162
:103A70000720FDF7C7FB06210820FDF7C3FB062141
:103A80000920FDF7BFFB06210A20FDF7BBFB06213D
:103A90001720FDF7B7FB06212820BDE80840FDF7F9
:103AA000B1BB000008B5FFF745FEFDF795FAFDF73D
:103AB0004FFDFDF73BFFFDF70FFEFFF7FDFDBDE8F6
:103AC0000840FFF769BD0000034611F8012B03F819
:103AD000012B002AF9D170471210121312110000A5
:103AE00053544D3332463F3F3F0000000120330026
:103AF0000010410101105A01031059010710310152
:103B000000000000E03A00083F000000130400003D
:103B1000383B00083F00000019040000423B000849
:103B20003F000000210400004C3B00083F00000063
:103B3000C02C00201C26002053544D333246343014
:103B4000780053544D3332463432780053544D3359
:103B50003246343436585800009600000000000009
:103B60000000000000000000000000000000000055
:103B70001915000805150008411500082D15000845
:103B8000391500082515000811150008FD14000856
:103B90004D15000800000000511600083D160008F1
:103BA0007916000865160008711600085D160008F1
:103BB0004916000835160008D51600080000000058
:103BC00001000000000000006D61696E000000004F
:103BD000E83B0008C82A0020C02C0020010000009B
:103BE000CD1F00080000000069646C650000000043
:103BF00002000000000000007D180008E518000821
:103C000040004000583100206831002002000000D0
:103C10000000000003000000000000002919000857
:103C200000000000100000007831002000000000BB
:103C300001000000000000004C34002001010200DF
:103C40004172647550696C6F740025424F41524453
:103C5000252D424C002553455249414C250000007A
:103C60008D230008F5220008E917000871230008D9
:103C700043000000783C000809024300020100C034
:103C800032090400000102020100052400100105B0
:103C90002401000104240202052406000107058214
:103CA000030800FF09040100020A000000070501E3
:103CB00002400000070581024000000012000000E1
:103CC000C43C0008120110010200004009124157D3
:103CD00000020102030100000403090425424F41D0
:103CE0005244250051696F54656B5A65616C6F745D
:103CF0004634323700303132333435363738394193
:103D000042434445460000000040000000400000DF
:103D10000040000000400000000001000000020020
:103D2000000002000000020000000200000002008B
:103D300000000200000002000040000000400000FF
:103D400000400000004000000000010000000200F0
:103D5000000002000000020000000200000002005B
:103D6000000002000000020000000000711A0008BC
:103D7000511D0008FD1D000840004000AC3400202B
:103D8000AC34002001000000BC34002080000000A2
:103D900040010000030000000001802A0000000034
:103DA000AAAAAAAA00010000FFFF0000000000006C
:103DB00000A00A001000000100000000AAAAAAA8A2
:103DC00010000001FFFF00000000000000000000E4
:103DD0000000004200000000AAAAAAAA00000041B8
:103DE000FFFF00000000000000000800600100006C
:103DF00000000000AAAAAAAA50010000FFFF0000CC
:103E0000000800000000000050001040000000000A
:103E1000AAAAAAAA00001040FFFF000000000000AC
:103E2000000000000000000000000000AAAAAAAAEA
:103E300000000000FFFF0000000000000000000084
:103E40000000000000000000AAAAAAAA00000000CA
:103E5000FFFF000000000000000000000000000064
:103E6000000000000A000000000000000300000045
:103E70000000000000000000000000000000000042
:103E80000000000000000000000000000000000032
:103E90000000000000000000FF0096000000000885
:103EA00004000000D83C00080000000000000000F2
:103EB0000000000000000000000000000000000002
:00000001FF
